:020000040800F2
:10000000503E00208502000835320008792500089E
:10001000CD310008B1040008793F0008000000005D
:10002000000000000000000000000000A501000822
:10003000E50600080000000001020008F73600088D
:100040009F0200089F0200089F0200089F0200080C
:100050009F0200089F0200089F0200089F020008FC
:100060009F0200089F0200089F0200089F020008EC
:100070009F0200089F0200089D050008A9050008CE
:100080009F0200089F0200089F0200089F020008CC
:100090009F0200089F0200089F0200089F020008BC
:1000A0009F0200089F0200089F0200089F020008AC
:1000B0009F02000800000000000000009F020008EE
:1000C0009F0200089F0200089F0200089F0200088C
:1000D0009F0200083D3F00089F0200089F020008A1
:1000E0009F0200089F0200080000000000000000BE
:1000F0000000000000000000000000000000000000
:10010000000000009F020008000000009F0200089D
:100110000000000000000000913700089F02000866
:100120009F0200089F0200089F0200089F0200082B
:100130009F02000800000000000000000000000016
:100140009F0200089F0200089F02000800000000B4
:100150009F0200089F0200089F0200089F020008FB
:100160009F0200089F0200089F0200080000000094
:100170009F0200089F02000800000000000000002D
:100180009F0200089F0200089F020008DFF810D0BD
:1001900000F024F9004800470D420008AFF300804A
:1001A000503E00202C4B1968086800F05AB880F3C4
:1001B0000988BFF36F8F4FF0000080F311887047FC
:1001C0000000000008480068006880F308884FF0CD
:1001D000000080F3148862B661B6BFF34F8FBFF39F
:1001E0006F8F00DF00BF00BF08ED00E0DFF80C00FC
:1001F000016841F470010160704700BF88ED00E0C4
:10020000EFF30980BFF36F8F134B1A681EF0100FC6
:1002100008BF20ED108A20E9F04F106009B44FF0BC
:10022000500080F31188BFF34F8FBFF36F8F05F03D
:1002300083F94FF0000080F3118809BC1968086841
:1002400000F014B81EF0100F08BF00F014B880F3CF
:100250000988BFF36F8F7047AC000020EFF3058073
:10026000704730C8B0E8C04FFFF7A1BF30C8B0E852
:10027000C04FFFF7E7BFB0EC088AB0EC08CAFFF741
:10028000E6BF00000648804706480047FEE7FEE755
:10029000FEE7FEE7FEE7FEE7FEE7FEE7FEE7FEE736
:1002A000813700088D0100082DE9F05F0546002028
:1002B00092469B4688460646814640241BE02846D7
:1002C00041464746224600F079F853465A46C01A3E
:1002D000914110D311461846224600F060F82D1ABD
:1002E00067EB01084F4622460120002100F057F835
:1002F00017EB00094E41201EA4F10104DFDC484643
:1003000031462A46434600F000B830BCBDE8C09FE5
:1003100040EA01039B0703D009E008C9121F08C087
:10032000042AFAD203E011F8013B00F8013B521E07
:10033000F9D27047D2B201E000F8012B491EFBD27E
:1003400070470022F6E710B513460A4604461946E0
:10035000FFF7F0FF204610BD30B5044600200346ED
:1003600000E05B1C934203D2E05CCD5C401BF8D004
:1003700030BD30B50B46014600202022012409E0A3
:1003800021FA02F59D4205D303FA02F5491B04FA4E
:1003900002F52844151EA2F10102F1DC30BD202A2D
:1003A00004DB203A00FA02F1002070479140C2F1CC
:1003B000200320FA03F3194390407047202A04DBFE
:1003C000203A21FA02F00021704721FA02F3D040CE
:1003D000C2F120029140084319467047064C074D70
:1003E00006E0E06840F0010394E807009847103405
:1003F000AC42F6D3FFF7CEFE44600008646000080C
:1004000030B58C1810F8012B12F00F0301D110F841
:10041000013B120906D110F8012B03E010F8015B33
:1004200001F8015B5B1EF9D101E001F8013B521EAE
:10043000FBD1A142E6D3002030BD00002DE9F04100
:100440009AB00646A1F11005684602F0A5F900240D
:100450004FF4007811E004F50070854201D9474659
:1004600000E02F1B31193A461048FFF751FF3A467A
:100470000E49684602F015FD3C44AC42EBD3694698
:1004800016A802F061F9002216A970198B5C845C31
:10049000A34203D1521C102AF8D301E0102A03D33F
:1004A00001201AB0BDE8F0810020FAE750020020D8
:1004B000FEE730B5002307E001EB830405682468FC
:1004C0004FEA34442C605B1CB3EB520FF4D3D207D9
:1004D00003D0026831F8231011800068006830BD35
:1004E00070B500230CE001EB83042588A6786DBA73
:1004F0002D04E47845EA06252543046825605B1C45
:10050000B3EB920FEFD394071BD002F00304012C3E
:1005100003D1066811F823503570022C05D101EB88
:1005200083040568248864BA2C80D243920708D1DA
:1005300001EB830103680A8852BA1A80026889783D
:1005400011700068006870BD70B54FF480752A4660
:100550000F491048FFF7DCFE0F4C20680088A0F51B
:100560002541A53912D0FF2229460A48FFF7E2FEAD
:1005700000F07AF920684BF6BB31A0F8FC1000219E
:1005800020F8EC1F4180416002F0AAFF002070BDFE
:10059000000001084801002040000020014800F050
:1005A00069BA0000A40D0020014800F063BA000001
:1005B0005C0D002030B590F8444004F01C05012487
:1005C000AC40056C6C60046863608368102B036842
:1005D00003D099600068C26030BD9A600068C16055
:1005E00030BD00007FB53D4C82784125A27030F8C7
:1005F000031F49BA8378090441EA0321C3781943E8
:1006000000918188837949BA090441EA0321C379B9
:10061000194301910189837A49BA090441EA032106
:10062000C37A194302918189837B49BA090441EA5B
:100630000321C37B19430391017C437C03EB01211C
:10064000837CC07C03EB012100EB0123A361E088E4
:10065000E1680D54401C80B200250D54401C80B24E
:10066000E080012A01D0062203E0B3F5803F02D9E1
:1006700002220A5404E001F0A1FFE088E1680D5471
:10068000401CE080E188E06801224554491C89B2A1
:100690004554491C89B24254491C89B21022455420
:1006A000491CE18069460E48FFF756FE50B10C48E0
:1006B0000099016001994160029981600399C160CC
:1006C000A560A580A188E088E2680B0A1354401C4D
:1006D00080B21154401CE0807FBD00005400002017
:1006E000500A0020704770B500231C4611E011F835
:1006F0002350055531F823502E0A05196E7051F814
:100700002360360CAE7051F823605B1C360EEE7021
:10071000241D9442EBD370BD72B6FEE7144A107FDD
:100720001449012801D003280FD10B6823F400736A
:100730000B600B6843F400630B600B6823F40063E9
:100740000B600B6843F400730B60022801D0032890
:100750000BD1086840F480500860086820F480508D
:100760000860086840F480600860002010777047D7
:100770008800002000200240C107054803D04169DD
:1007800041F004014161416941F4803141617047A8
:100790000020024008494A69C0B222F47E7242EA4F
:1007A000C0004861486940F002004861486940F46F
:1007B000803048617047000000200240054910B5B4
:1007C0004C6944F001044C610260BFF36F8F4360D9
:1007D00010BD000000200240094B10B55C694022AA
:1007E00044F480245C61EFF3108372B610C910C02A
:1007F000521E12F0FF02F9D183F3108810BD0000E1
:100800000020024070B5044600F000FC0646134D7F
:1008100008E0601C06D000F0F9FB801BA04201D369
:10082000032070BD2869C003F3D428690C4908402F
:100830000CD00C494A6802434A60810F01D0A96973
:10084000A961810000D02861012070BD2869C0071E
:1008500001D001202861002070BD0000002002406E
:10086000FAC302008800002004484AF2A55100683B
:100870000180012181700221C17070474000002079
:100880000549884202D2A0F1006002E002494942D3
:100890000844C00A7047000000000408F0B505468F
:1008A00000201F2301265B1E05D303F01F0706FA55
:1008B00007F40C42F7D07AB1082A09D0102A04D0E4
:1008C000182A07D1072B05D206E0082B02D203E035
:1008D000102B01D30120F0BD0028FCD12B685961F9
:1008E00029688B6823F0180313438B60F0BD70B543
:1008F000044600200223637723689D6845F00105C4
:100900009D60236A012B0FD0022B11D0032B12D133
:10091000002304E0256851F8230028605B1C934203
:10092000F8D32068006806E02046FFF7D9FD02E012
:100930002046FFF7BEFD0121617770BD10B50400B0
:1009400010D0607F20B900202077204600F030F8DA
:1009500002206077207938B1D4E902122046FFF7EF
:100960009DFF48B1012010BD2168104848612068F2
:10097000816821F0180181606079A0B12069216847
:10098000086120688168626921F06001114381601B
:1009900020688168A26921F08001114381600120F3
:1009A0006077002010BD4FF0FF30E8E7B71DC104AD
:1009B00008B500680649884208D10648816C41F4B0
:1009C00080518164806C00F48050009008BD00006C
:1009D000003002400010024010B590F825100022AF
:1009E000022905D00421C16380F82420012010BD14
:1009F00001680B6823F00E030B6001680B6823F09D
:100A000001030B6090F84410012401F01C0304FA68
:100A100003F1036C596080F8254080F824201046CB
:100A200010BD10B590F825100024022903D0042130
:100A3000C16301241AE001680A6822F00E020A600C
:100A400001680A6822F001020A6090F8441001234C
:100A500001F01C0203FA02F1026C516080F82530AB
:100A6000002180F82410816B01B18847204610BD19
:100A7000C06B7047F0B4016C0B6801680A6890F8AD
:100A80004440042504F01C0405FA04F61E4211D06B
:100A900056070FD50A68920603D40A6822F00402AA
:100AA0000A6090F8441001F01C018D40016C4D600B
:100AB000016B1DE0022606FA04F71F424FF0000CFE
:100AC0004FF0010518D0970716D50A68920605D48D
:100AD0000A6822F00A020A6080F8255090F8441053
:100AE00001F01C018E40016C4E6080F824C0C16A88
:100AF00000291AD0F0BC08470826A6401E4214D090
:100B0000120712D50A6822F00E020A6090F844100B
:100B1000026C01F01C0105FA01F15160C56380F817
:100B2000255080F824C0416BE2E7F0BC704700001C
:100B300070B568B1334C01681423334AA14209D21D
:100B4000324C0C44B4FBF3F39B00C0E910230BE0E0
:100B5000012070BD2B4C64420C44B4FBF3F39B00AA
:100B60004364284B083B0364022380F825300C685B
:100B700047F6F0739C43D0E902352B43D0E9045685
:100B800035432B4385692B43C5692B43056A2B43AA
:100B900023430B608168B1F5804F29D0016C0F238E
:100BA000914212D152F8A81F90F8444004F01C045E
:100BB000A3409943116090F84430416803F01C034E
:100BC000994013681943116012E00E49A0310A6878
:100BD00090F8444004F01C04A3409A430A6090F843
:100BE0004430426803F01C039A400B681A430A60C1
:100BF0000021C163012280F8252080F824100846D6
:100C000070BD00000804024000000240F8FFFDBF74
:100C100070B5044690F82400002501280CD001206E
:100C200084F8240094F825600020012E06D084F872
:100C300024000225284670BD022070BD022684F8DB
:100C40002560E0632068066826F0010606602046FD
:100C5000FFF7B0FC206B00282068016802D041F04B
:100C60000E0106E021F0040101602068016841F0F6
:100C70000A0101602068016841F001010160D9E7C3
:100C80002DE9F05F044632488946017801290CD0ED
:100C90000125804605704CF2503B5846FFF7B2FDE7
:100CA00006004FF0000A03D04EE0022000F054B8D6
:100CB00051464046C8F804A0264F3A6892050AD526
:100CC0003968490505D5396821F480613960032107
:100CD00009E0057708E03A68520504D5396821F43F
:100CE00080613960022101772068012807D04FF028
:100CF000FF31C9F8001040F2FA3BA5681DE06068BA
:100D0000FFF73AFD5846FFF77DFD0646786920F06B
:100D10000400786116E028466168FFF73BFD4CF25D
:100D20005030FFF76FFD0600786920EA0B0078610C
:100D300002D0C9F8005005E06D1CD4E90201084456
:100D4000A842E8D8FFF7EAFC88F800A03046ADE7F3
:100D5000880000200020024030BCBDE8C09F000099
:100D60000348416941F000414161002070470000A3
:100D7000002002402DE9FF5F254F0546002438780A
:100D800091469B46012809D0012038704CF2503022
:100D9000FFF738FD0600A24604D035E0022004B07B
:100DA00000F03AB85046C7F804A0DFF86880D8F8D9
:100DB0000010490506D5D8F8001021F48061C8F864
:100DC00000100220387725B1012D09D0022D07D05F
:100DD0000DE04A465B460198FFF7F0FC012406E06F
:100DE00049460198FFF7F8FC022D00D16C044CF243
:100DF0005030FFF707FD064624B1D8F81410A14380
:100E0000C8F81410FFF78AFC87F800A03046C6E740
:100E1000880000200020024030BCBDE8C09F0000D8
:100E2000064900204A69002A07DA054A8A60054A0D
:100E30008A604969002900DA0120704700200240D9
:100E400023016745AB89EFCD2DE9F84FDFF880919D
:100E50000022A9F1040B03274FF00F0C09F1040A3B
:100E6000ABF1040EACE0012595402B4073D00C791A
:100E700004F00304012C01D0022C15D18668540023
:100E800007FA04F826EA0806D1F80C8008FA04F8F4
:100E900048EA0608C0F808804468AC430D79C5F3F9
:100EA00000159540254345600C79E443A40708D01C
:100EB000C568540007FA04F6B5438E68A6402E4371
:100EC000C6600C7904F00304022C11D1D40800EBA5
:100ED0008406356A5407E40E0CFA04F825EA08057E
:100EE000D1F8108008FA04F848EA0508C6F820800E
:100EF0000568540007FA04F6B5430E7906F00306B8
:100F0000A6402E4306604C6814F4403F57D0314C45
:100F1000256E45F001052566246E22F0030504F0D8
:100F2000010400942C4C05EB0408D8F808509407F1
:100F3000260F0CFA06F4A543B0F1904F04D0274CCD
:100F4000A04203D1012412E0002410E0244CA0426E
:100F500002D102240BE032E0224CA04201D1032452
:100F600005E0214CA04201D1042400E00724B44054
:100F70002C43C8F80840D9F800404D464E689C43C1
:100F8000F60200D51C432C60DAF8004055464E6846
:100F90009C43B60200D51C432C60DBF800405D4644
:100FA0004E689C43B60300D51C432C60DEF800401D
:100FB00075464E689C43F60300D51C432C60521CBA
:100FC0000B6833FA02F47FF44EAF00F00FB8000064
:100FD00008040140001002400000014000040048E5
:100FE00000080048000C00480010004818BCBDE88C
:100FF000E08F426921EA02030A4043EA024181612B
:1010000070470AB18161704781627047014880680A
:10101000704700007C00002002488168027811447B
:10102000816070477C00002010B50024032000F090
:101030009FF80F2000F008F808B1012401E000F04B
:101040004FF8204610BD000030B505461F4887B058
:10105000816D41F010018165806D06A900F01000DE
:101060000590684600F0D4FA0398B0B100F0F0FAA9
:1010700040001749174AB0FBF1F11748491E0260BA
:10108000416040F2E7320021C0E9032181608161C3
:1010900000F0FDFD040003D015E000F0D9FAE8E708
:1010A0000D4800F027FE04000DD1362000F032F884
:1010B000102D07D200222946362000F039F80748C3
:1010C000056000E0012407B0204630BD001002405A
:1010D00040420F0000100040EC0D00208000002076
:1010E0000B4882B0016E41F001010166016E01F012
:1010F00001010091816D41F080518165806D002278
:1011000000F0805000900F21901E02B000F010B847
:1011100000100240002809DB00F01F02012191406D
:101120004009800000F1E020C0F800117047000085
:10113000F0B40E4B1B68C3F30223C3F10704042C65
:1011400000D904241D1D072D01D2002300E0DB1E61
:10115000012606FA04F56D1E0D409D409E40761E48
:10116000164045EA0601F0BC02F064BF0CED00E059
:10117000064A00F0070110684FF6FF03184040EAE6
:101180000120034908431060704700000CED00E0A7
:101190000000FA051649B0F5007F0868C0F3412049
:1011A00009D0022805D0086820F4C06040F48060AF
:1011B0000860002070470128FBD0086820F4C06058
:1011C00040F4007008600B483222006850430A4A1D
:1011D000B0FBF2F0401C00E0401E4A69520501D508
:1011E0000028F9D148694005E3D503207047000085
:1011F00000700040A800002040420F000248006834
:1012000000F4C06070470000007000402DE9F84F06
:10121000044600250088A64E2F46000515D5606CB3
:1012200060B1B0F5000F04D0B0F5400F2BD0012510
:101230000AE0F06840F48030F06024E00021201DD6
:1012400001F0FAFF05001ED02F462068800365D507
:10125000B06D4FF00009C00009D4B06D40F080506F
:10126000B065B06D4FF0010900F080500090DFF8DC
:1012700044A2DAF8001041F48071CAF80010FFF7B8
:10128000C5FE804610E0D6F88800616C20F440006E
:101290000843C6F88800D8E7FFF7B8FEA0EB0800BF
:1012A000022801D9032531E0DAF80000C005F3D5A2
:1012B00065BBD6F8900010F4407014D0A16D814247
:1012C00011D0D6F89000D6F8901020F4407041F478
:1012D0008031C6F89010D6F8901021F48031C6F80D
:1012E0009010C6F89000C0074ED0FFF78FFE8046E2
:1012F00041F2883A05E0FFF789FEA0EB080151456D
:10130000D0D8D6F890008007F5D5EDB32F46B9F1C7
:10131000000F03D0B06D20F08050B0652078C0077A
:1013200007D0D6F88800216A20F003000843C6F8E9
:1013300088002078800707D5D6F88800616A20F0F9
:101340000C000843C6F888002078400707D5D6F877
:101350008800A16A20F030000843C6F88800207891
:10136000800607D5D6F88800E16A20F4406008437B
:10137000C6F888002088800509D5D6F88800E16B7A
:1013800020F44020084300E044E0C6F888002088AC
:10139000400507D5D6F88800216C20F4401008439A
:1013A000C6F888002078400607D5D6F88800216B5B
:1013B00020F440500843C6F888002078000607D57E
:1013C000D6F88800616B20F440400843C6F88800D6
:1013D0002088C00507D5D6F88800A16B20F44030DE
:1013E0000843C6F8880020684FF0006500034FF0FE
:1013F000806820D5D6F88800A16C20F040600843B2
:10140000C6F88800A06CA8420DD1F06840F48010A6
:10141000F06010E0D6F89000A16D20F44070084311
:10142000C6F8900073E7404505D10121201D01F069
:1014300003FF00B107462068400317D5D6F888009F
:10144000E16C20F040600843C6F88800E06CA842D8
:1014500004D1F06840F48010F06007E0404505D109
:101460000121201D01F0E8FE00B10746208840045C
:1014700011D5D6F88800216D20F040500843C6F8F9
:101480008800206DB0F1805F05D10221201D01F0A0
:10149000D3FE00B107462088000406D556F8880F11
:1014A000616D20F0804008433060384600F004B899
:1014B000001002400070004018BCBDE8E08F000042
:1014C0002DE9F0470D46040071D0DFF83081D8F8DF
:1014D000000000F00700A8420CD2D8F8001021F05C
:1014E00007012943C8F80010D8F8000000F00700F1
:1014F000A8425CD12078424E80070AD5A068B16826
:1015000001F0F001884204D9B16821F0F0010143F3
:10151000B1602078C0072BD06068032811D0022862
:1015200012D0316898B14905002940DAB16821F03C
:1015300003010143B160FFF769FD074641F28839B5
:101540000FE031688901EFE731688903ECE789072B
:10155000EAE7FFF75BFDC11B494502D90320BDE85F
:10156000F087B068616800F00C00B0EB810FF0D13B
:10157000207880070AD5A068B16801F0F0018842A0
:1015800004D2B16821F0F0010143B160D8F8001035
:10159000404601F00701A9420BD9016821F007017B
:1015A00029430160006800F00700A84201D0012033
:1015B000D5E72078400705D5B068E16820F4E06001
:1015C0000843B0602078000706D5B068216920F490
:1015D000605040EAC100B06000F05EF8B168094AAE
:1015E000C1F30311515C01F01F01C84006490860B6
:1015F00006480068BDE8F047FFF726BD002002401E
:1016000000100240E45F0008A800002080000020D5
:101610000F2202600C4A936803F00303436093684F
:1016200003F0F0038360936803F4E063C36092689F
:101630004FF4E06303EAD20202610448006800F05C
:1016400007000860704700000010024000200240C0
:101650000548064900688968054AC1F30221515CC2
:1016600001F01F01C8407047A80000200010024090
:10167000246000080548064900688968054AC1F3E6
:10168000C221515C01F01F01C8407047A800002032
:10169000001002402460000870B5254B002210465F
:1016A0009968DC6811F00C0104F00306214C4FEA44
:1016B000640508D00C2904D0042931D0082931D080
:1016C00010E0012E10D11A68120704D4D3F8942028
:1016D000C2F3032202E01A68C2F30312164E56F850
:1016E0002220D9B10C2918D1D86800F003000228B3
:1016F0001AD003281AD01046D968DA68C1F302114B
:10170000C2F306224243491CB2FBF1F0D968C1F38F
:101710004161491C4900B0FBF1F070BD104670BD3D
:10172000204670BD284670BD2046E5E72846E3E721
:10173000001002400024F400F45F00082DE9F84393
:1017400004006FD0F64EB06800F00C05F06800F0B1
:1017500003072078C00664D575B10C2D01D1012F87
:101760000AD0A0690028306879D040F001003060CC
:10177000FFF74CFC80465CE03068800702D5A0692A
:101780000028DED0216A3068000703D5306800F0F9
:10179000F00004E0D6F89400F02202EA1010814232
:1017A00016D9084601F0DCFD00283BD1306840F036
:1017B000080030603068216A20F0F0000843306093
:1017C0007068E16920F47F4040EA0120706016E013
:1017D000306840F0080030603068216A20F0F00086
:1017E000084330607068E16920F47F4040EA0120DE
:1017F000706025B9206A01F0B3FD0028D5D1FFF74C
:101800004BFFB168C74AC1F30311515C01F01F01DE
:10181000C840C5490860C5480068FFF715FC0028A6
:101820007ED12CE0C6E0FFF7F1FBA0EB0800022818
:1018300077D830688007F6D5306840F0080030600F
:101840003068216A20F0F000084330607068E16978
:1018500020F47F4040EA0120706010E0FFE720F0B4
:1018600001003060FFF7D2FB804605E0FFF7CEFBBA
:10187000A0EB08000228DBD830688007F6D4207877
:10188000C00740D0082D18D00C2D01D1032F14D043
:101890006068B0F5803F17D0B0F5A02F306817D042
:1018A00020F480303060306820F480203060606840
:1018B000E0B1FFF7ABFB804614E03068800322D52F
:1018C0006068002876D01EE0306840F48030EDE794
:1018D00040F480203060F7E7FFF798FBA0EB0800AA
:1018E0006428A5D830688003F6D50CE0FFF78EFB9E
:1018F000804605E0FFF78AFBA0EB0800642897D834
:1019000030688003F6D42078800739D5042D11D0B3
:101910000C2D01D1022F0DD0E0680028306801E0C5
:10192000A0E1FBE01DD040F480703060FFF76EFB5B
:1019300007460BE0306840050BD5E0680028C1D0B1
:1019400007E0FFF763FBC01B022894D8306840050E
:10195000F7D57068217C20F0F85040EA0160706093
:101960000EE020F480703060FFF750FB074604E083
:10197000FFF74CFBC01B0228B3D830684005F7D4F2
:101980002078000728D560690028D6F8940012D086
:1019900040F00100C6F89400FFF738FB074604E06A
:1019A000FFF734FBC01B02289BD8D6F894008007B1
:1019B000F6D511E027E120F00100C6F89400FFF70A
:1019C00025FB074604E0FFF721FBC01B022888D84F
:1019D000D6F894008007F6D42078400765D5B06D1E
:1019E0004FF00008C00009D4B06D40F08050B065E1
:1019F000B06D4FF0010800F0805000904C48016835
:101A0000C90511D40168814641F480710160FFF776
:101A1000FDFA074604E0FFF7F9FAC01B02287DD85B
:101A2000D9F80000C005F6D5A068012815D0052812
:101A3000D6F8900016D020F00100C6F89000D6F835
:101A4000900020F00400C6F89000A06841F28839A8
:101A5000B8B1FFF7DBFA07460EE0D6F8900040F089
:101A60000100F0E740F00400C6F89000F5E7FFF74A
:101A7000CDFAC11B494551D8D6F890008007F6D55C
:101A80000CE0FFF7C3FA074604E0FFF7BFFAC11BFB
:101A9000494543D8D6F890008007F6D4B8F1000F36
:101AA00003D0B06D20F08050B0652078800627D537
:101AB000606A0028D6F8980011D040F00100C6F8FE
:101AC0009800FFF7A3FA074604E0FFF79FFAC01B50
:101AD000022823D8D6F898008007F6D510E020F029
:101AE0000100C6F89800FFF791FA074604E0FFF7F7
:101AF0008DFAC01B022811D8D6F898008007F6D4BA
:101B0000A06AE8B3022815D00C2D7CD0306820F0F4
:101B100080703060FFF77AFA0446A5E0A1E000008B
:101B200000100240E45F0008A800002080000020B0
:101B300000700040F068E26A00F00301914228D191
:101B4000216B00F0700209011039914221D1626BC2
:101B500000F4FE41B1EB022F1BD194F8382000F0C5
:101B60007841B1EBC26F14D1A18F00F4C0024908D3
:101B70004905A1F5001191420BD194F8401000E005
:101B800069E04908490600F0C060A1F10071814296
:101B90004AD00C2D71D0306840016ED4306820F0EE
:101BA00080703060FFF732FA054604E0FFF72EFA46
:101BB000401B022855D830688001F7D4F4E90B01A6
:101BC0006FF00F0202EB01110843218A5204490809
:101BD00002EB4151A26841EA02210843217D4FF006
:101BE0007E42490802EB41610843217B40EAC16023
:101BF000F168234A11400843F060306840F080707B
:101C00003060F06800E038E040F08070F060FFF78E
:101C1000FDF9044604E0FFF7F9F9001B022820D87B
:101C200030688001F7D526E03068800123D4306821
:101C300040F080703060F06840F08070F060FFF736
:101C4000E5F9044604E0FFF7E1F9001B022808D893
:101C500030688001F7D50EE0FFF7D8F9001B0228A5
:101C600002D90320BDE8F88330688001F4D4F0681D
:101C700004490840F0600020F4E70120F2E700008A
:101C80008C809D01FCFFEEFE70477047704710B5D9
:101C9000040003D094F83D0010B107E0012010BD0E
:101CA000002084F83C00204600F022F8022084F84E
:101CB0003D00211D206801F071FD012084F84800DD
:101CC00084F83E0084F83F0084F8400084F8410026
:101CD00084F8420084F8430084F8440084F8450006
:101CE00084F8460084F8470084F83D00002010BDC9
:101CF0007047000090F83D10012901D00120704785
:101D0000022180F83D100168CA6842F00102CA60F1
:101D100000680B49884205D0B0F1804F02D00949D4
:101D2000884207D18168084A1140062906D0B1F5DA
:101D3000803F03D0016841F001010160002070473D
:101D4000002C01400040014007000100704770B5C1
:101D50000446006801694FF00005C943890715D49E
:101D6000C168C943890711D4E91E016101202077A8
:101D7000206880698007204602D0FFF7E7FF04E073
:101D800000F0A7F8204600F0A5F825772068016943
:101D9000C943490717D4C168C943490713D46FF031
:101DA00004010161022020772068806910F4407FDF
:101DB000204602D0FFF7CAFF04E000F08AF8204670
:101DC00000F088F8257720680169C943090716D40F
:101DD000C168C943090712D46FF0080101610420EA
:101DE00020772068C0698007204602D0FFF7AEFF49
:101DF00004E000F06EF8204600F06CF825772068CB
:101E00000169C943C90617D4C168C943C90613D4B7
:101E10006FF010010161082020772068C06910F47C
:101E2000407F204602D0FFF791FF04E000F051F818
:101E3000204600F04FF8257720680169C943C9079B
:101E400008D1C168C943C90704D1891E0161204670
:101E500000F042F820680169C943090609D4C16845
:101E6000C943090605D46FF0800101612046FFF7E0
:101E70000CFF20680169C943C90509D4C168C94379
:101E8000090605D46FF4807101612046FFF7FCFE5E
:101E900020680169C943490609D4C168C943490694
:101EA00005D46FF040010161204600F01FF8206862
:101EB0000169C94389060BD4C168C943890607D49F
:101EC0006FF0200101612046BDE87040FFF7DEBEE3
:101ED00070BD70477047000000680349884201D117
:101EE000FFF79AB870470000001000407047704735
:101EF000704770B50446806FE66F216889684FF0BF
:101F00001005090618D5212816D12068083050E898
:101F1000001F21F0800140E80012002AF5D1E06E98
:101F200038B1FEF759FD20B1E06EFEF7A1FD202883
:101F300021D0204601F043FE20688068400618D575
:101F4000222E16D12068083050E8001F21F04001F1
:101F500040E80012002AF5D1206F38B1FEF73CFDB1
:101F600020B1206FFEF784FD202804D0204601F028
:101F700001FE002070BDC4F88050032070BD704782
:101F80002DE9F04102680446D0691168966840F670
:101F90000F0318424FF0000505D183067ED58B064E
:101FA0007CD5616E1BE1994F06F001030F401F4382
:101FB00074D0C70709D0CF0507D501271762D4F819
:101FC000802042F00102C4F8802082070AD5F2077F
:101FD00008D0276802223A62D4F8802042F0040236
:101FE000C4F8802042070AD5F20708D026680422E8
:101FF0003262D4F8802042F00202C4F88020020746
:102000000CD501F020021A4308D0236808221A6276
:10201000D4F8802042F00802C4F8802002050BD5D5
:102020004A0109D523684FF400621A62D4F880206F
:1020300042F02002C4F88020D4F88020002A35D055
:10204000800605D5880603D5616E09B1204688470C
:10205000D4F8800021688968490602D410F0280F5E
:1020600026D0204601F086FD2068806840061AD5FB
:102070002068083050E8001F21F0400140E80012BD
:10208000002AF5D1206F70B161498163206FFEF79E
:10209000C8FC00280AD0206F816B01E00EE02046CA
:1020A000BDE8F04108472046FFF769FFBDE8F08131
:1020B0002046FFF764FFC4F88050F7E7276E20231F
:1020C000012F7BD1C70679D5CF0677D510201062B6
:1020D00020688068400641D5216F08684068000488
:1020E000000CE3D0B4F858208242DFD9A4F85A009B
:1020F0000868006880062AD4206850E8001F21F490
:10210000807140E80012002AF6D12068083050E8BB
:10211000001F21F0010140E80012002AF5D12068DB
:10212000083050E8001F21F0400140E80012002A6A
:10213000F5D1E3672566206850E8001F21F0100103
:1021400040E80012002AF6D1206FFEF745FCB4F8F3
:102150005800B4F85A10401A81B22AE0B4F8580076
:10216000B4F85A10401A81B2B4F85A0000289DD031
:1021700000299BD0206850E8002F22F4907240E89C
:102180000026002EF6D12068083050E8002F22F0FB
:10219000010240E80026002EF5D1E367256665665A
:1021A000206850E8002F22F0100240E80023002BA6
:1021B000F6D12046FFF79BFE78E7FFE7C70209D577
:1021C000760207D54FF4801010622046BDE8F0413A
:1021D000FFF78EBE020606D50A0604D5A16E0029B9
:1021E0007FF45DAF62E74006E6D54806E4D52046B9
:1021F000016851E8002F22F0400241E80024002C41
:10220000F6D18367856600F0B5F94FE72001000439
:102210002D3A000810B5040002D0A06F10B107E0FD
:10222000012010BD002084F87400204600F026F83C
:102230002420A0672068016821F001010160204688
:1022400001F0CAFC0128ECD0606A10B1204601F010
:102250005BFB2068416821F49041416020688168FF
:1022600021F02A0181602068016841F001010160CC
:102270002046BDE8104001F0ABBB00002DE9F04363
:102280009DB00446142117A8FEF75BF85C21684650
:10229000FEF757F846492068464E022700254FF0C2
:1022A00003084FF0070988425BD101200090089590
:1022B0006846FEF7ABFF08B1FEF72EFA306E40F429
:1022C00080403066306E00F480401C90F06C40F02E
:1022D0000100F064F06C19AA00F001001C904FF4AA
:1022E000C060CDE9170782E8200317A94FF090409E
:1022F000FEF7AAFD314E30484FF080083060C6E945
:102300000175C6E903587561B561F56130463562FE
:10231000FEF70EFC08B1FEF7FFF92667B462274E00
:10232000254848361438E6E802071020A6E82101BF
:10233000224846F814594830B561F5613562FEF718
:10234000F7FB08B1FEF7E8F9E66600220521252033
:10235000B462FEF7EDFE2520FEF7DCFE1DB0BDE801
:10236000F08317498842F9D104200A950090684605
:10237000FEF74CFF08B1FEF7CFF9B06D40F48020B6
:10238000B065B06D00F480201C90F06C40F004004B
:10239000F064F06C19AA00F004001C903020CDE924
:1023A000170782E8200317A90648FEF74DFDD5E779
:1023B0000038014000100240580002405C0D00202F
:1023C000004800400008004830B4C36F202B20D1E3
:1023D000E1B1DAB190F87430012B1AD0012380F802
:1023E0007430002303660C4C0368A3420BD05B6877
:1023F0001B0208D5036853E8004F44F0806443E8AB
:102400000045002DF6D130BC01F0E4BC012030BC09
:1024100070470220FBE700000080004070477047D3
:102420002DE9F8430446806F1F4615460E462028C6
:102430004ED1CEB1C5B194F87400012848D0012026
:1024400084F874004FF00008C4F880802120A06751
:10245000FEF7DCFDA4F850508146A4F85250A06865
:10246000B0F5805F03D004E00120BDE8F883206967
:1024700020B13546002684F8748010E00025FAE784
:102480008021204601F0F8FCB8B9C5B115F8010B60
:1024900021680885B4F85200401EA4F85200B4F830
:1024A00052004B464FF0000200970028E8D14FF051
:1024B0004001204601F0E0FC30B10320D5E736F8BA
:1024C000020BC0F30800E3E72020A0670020CCE760
:1024D0000220CAE770B50446806F202841D169B355
:1024E00062B394F8740001283BD0012084F8740092
:1024F000E164A4F85020A4F852200025C4F88050CC
:102500002120A067E06ED8B11749C162E16E17487B
:1025100013460863E16E16484863E06E85632668DB
:10252000E16C06F12802E06EFEF772FB40B110206C
:10253000C4F8800004F8745F20206060012070BD42
:1025400021684020086284F874502068083050E800
:10255000001F41F0800140E80012002AF5D1002060
:1025600070BD022070BD0000293B00086B3B0008D5
:10257000413A000870477047FEE7000070B50E4C06
:1025800000230126E260E38003780725402B05D174
:1025900043783BB1012B08D0022B09D01570E6809F
:1025A000E08870BDFEF71EF8FAE701F02DF9F7E7B5
:1025B00001F078F9F4E70000540000200448417865
:1025C000012903D0034901610121417070470000D6
:1025D0005400002000000308F0B585B0174D00241A
:1025E00004946C70164928690844B0F5803F02D302
:1025F000081705B0F0BDFEF713FC00942869FEF73C
:102600003FF9029001200190039004A96846FEF76B
:1026100037FB0C4E002406EBC400D0E900232869E8
:1026200000EBC4010020FEF7A5FB641C0746FF2C4D
:10263000F1DDFEF795FB3846DBE700005400002093
:102640000000FDF7500200202DE9F04F064687B04C
:1026500000202C4FCDE9040082467878DFF8A8905E
:102660000D464FF4006B012806D147E02749386931
:102670000844B0F5803F04D34FF0FF3007B000F0BE
:1026800047B87869D8464119414503D9C0F500617A
:102690008CB200E02C46484422463146FDF738FE15
:1026A0007869291B204426448DB27861404525D1A4
:1026B000FEF7B6FBCDF800A0D0463869FEF7E0F88B
:1026C000029001200190039005A96846FEF7D8FA10
:1026D000002409EBC400D0E90023386900EBC401F1
:1026E0000020FEF747FB641C0490FF2CF1DDFEF791
:1026F00037FB386900F50060C7E90408002DB5D143
:102700000498BBE754000020500200200000FDF7B1
:1027100030BCBDE8C08F000008490868084A104076
:10272000B0F1005F09D1012080F310884868054AA4
:10273000D061096881F308880047704700000208EB
:102740000000FE2F540000207CB50C4605460822F0
:1027500010316846FDF7C7FF208AC0F3C502382A4A
:1027600002D2C2F1380201E0C2F1780209492046E2
:1027700000F097FB08226946204600F092FB1022E9
:1027800021462846FDF7AFFF58220021204600F0E1
:10279000C9FB7CBD000000200021416101610549A9
:1027A0000160054941600349C94381600249C94349
:1027B000C16070470123456789ABCDEF2DE9F04F2C
:1027C00050F804BB002590E8580091B0EA464FF05D
:1027D00040092A46001F8F18121D97F80280B7F88B
:1027E00000C0FF7868F31F4C4CEA076C4AF825C01C
:1027F0006D1C4A45EFD303EA040126EA03021143A4
:10280000FE4A009D0A4405EB0B01114403EB716283
:1028100002EA030124EA02073943F94F3944019FD0
:102820003E44314402EB315101EA020623EA01073A
:102830003E43F44F3E44029F3C44344401EBF434A5
:1028400004EA010622EA04073E43EF4F3E44039F99
:102850003B44334404EBB32303EA040621EA0307B1
:102860003E43EA4F3E44049F3A44324403EB7262D3
:1028700002EA030624EA02073E43E54F3E44059F71
:102880003944314402EB315101EA020623EA0107DF
:102890003E43E04F3E44069F3C44344401EBF43455
:1028A00004EA010622EA04073E43DB4F3E44079F49
:1028B0003B44334404EBB32303EA040621EA030751
:1028C0003E43D64F3E44089F3A44324403EB726283
:1028D00002EA030624EA02073E43D14F3E44099F21
:1028E0003944314402EB315101EA020623EA01077F
:1028F0003E430A9FA6F524463C444F3E344401EB38
:10290000F43404EA010622EA04073E43C54F3E447C
:102910000B9F3B44334404EBB32303EA040621EA50
:1029200003073E43C04F3E440C9F3A44324403EBFE
:10293000726202EA030624EA02073E43BB4F3E44AA
:102940000D9F3944314402EB315101EA020623EA7A
:1029500001073E43B64F3E440E9F3C44344401EBD6
:10296000F43404EA010622EA04073E43B14F3E4430
:102970000F9F3B44334404EBB32303EA010624EAEC
:1029800001073E43AC4F3E44019F3A44324403EBBF
:10299000F26202EA040623EA04073E43A74F3E44DC
:1029A000069F3944314402EBF15101EA030622EA61
:1029B00003073E43A24F2B443E440B9F3C44344408
:1029C00001EBB44404EA020621EA02073E439D4FAC
:1029D0003E44334404EB333303EA010624EA01079F
:1029E0003E43994F3E44059F3A44324403EBF26222
:1029F00002EA040623EA04073E43944F3E440A9F3A
:102A00003944314402EBF15101EA030622EA03079B
:102A10003E438F4F3E440F9F3C44344401EBB4444B
:102A200004EA020621EA02073E438A4F3E44049F1D
:102A30003B44334404EB333303EA010624EA010741
:102A40003E43854F3E44099F3A44324403EBF262D1
:102A500002EA040623EA04073E43804F3E440E9FE9
:102A60003944314402EBF15101EA030622EA03073B
:102A70003E437B4F3E44039F3C44344401EBB4440B
:102A800004EA020621EA02073E43764F3E44089FCD
:102A90003B44334404EB333303EA010624EA0107E1
:102AA0003E43714F3E440D9F3A44324403EBF26281
:102AB00002EA040623EA04073E436C4F3E44029FA9
:102AC0003944314402EBF15101EA030622EA0307DB
:102AD0003E43674F3E44079F3C44344401EBB444BB
:102AE00004EA020621EA02073E43624F3E440C9F7D
:102AF0003B443344059E04EB3333164483EA04021B
:102B00005D4F4A403A443244089E03EB32720E4411
:102B100082EA0301594F61403944314402EB715656
:102B20000B99574F0C4486EA02015940394421441D
:102B300006EB31440E99534F0B4484EA0601514091
:102B400039441944019B04EB7121134481EA0402C6
:102B50004D4F72403A441A44049B01EB32721E44BA
:102B600082EA0103494F63403B44334402EB73560E
:102B7000079B474F1C4486EA02034B403B442344D7
:102B80000A9C06EB33430C4483EA0601414F514053
:102B9000394421440D9C03EB7121144481EA030262
:102BA00072403D4F2E443A44224401EB327282EA95
:102BB00001043A4F5C403C443444039E02EB74549D
:102BC0001E4484EA0203364F4B403B443344069E86
:102BD00004EB33430E4483EA0401324F514039443D
:102BE0003144099E03EB7121164481EA03022E4F02
:102BF00062403A44324401EB327257E078A46AD71B
:102C000056B7C7E8DB702024EECEBDC1AF0F7CF510
:102C10002AC68747134630A8019546FDD898806993
:102C2000AFF7448BBED75C892211906B937198FDEE
:102C30008E4379A62108B44962251EF640B340C0F0
:102C4000515A5E26AAC7B6E95D102FD65314440226
:102C500081E6A1D8C8FBD3E7E6CDE121D60737C38B
:102C6000870DD5F4ED145A4505E9E3A9F8A3EFFC67
:102C7000D9026F678A4C2A8D4239FAFF81F6718733
:102C800022619D6D0C38E5FD44EABEA4A9CFDE4B60
:102C9000604BBBF670BCBFBEC67E9B28FA27A1EA7C
:102CA0008530EFD4051D880439D0D4D90C9E684FE7
:102CB000264482EA01045C403C4434440F9E02EB0B
:102CC00074541E4484EA0203624F4B403B44334435
:102CD000029E04EB33430E4483EA04015E4F5140ED
:102CE0003944314403EB7121154461EA04025B4E1F
:102CF0005A4032442A44079D01EBB262254462EAFD
:102D00000304574E4C4034442C440E9D02EBB45403
:102D10001D4464EA0103534E534033442B44059D44
:102D200004EB73430D4463EA02014F4E61403144AA
:102D300029440C9D03EBF121154461EA04024B4E3A
:102D40005A4032442A44039D01EBB262254462EAB0
:102D50000304474E4C4034442C4402EBB4550A9CC7
:102D60001C4465EA01035340424E3344234405EBBF
:102D70007344019B404E0B4464EA020169403144B4
:102D8000194404EBF12308993C4E0A4463EA050117
:102D90006140314411440F9A03EBB161154461EA7B
:102DA0000402374E5A4032442A44069D01EBB25287
:102DB000254462EA0304334E4C4034442C440D9DB8
:102DC00002EB74441D4464EA01032F4E5340334424
:102DD0002B44049D04EBF3230D4463EA02012B4EC4
:102DE0006140314429440B9D03EBB161154461EA14
:102DF0000402274E5A4032442A44029D01EBB2524B
:102E0000254462EA0304234E4C4034442C44099D7B
:102E100002EB74441D4464EA01031F4E53403344E3
:102E20002B44056804EBF3232944016041681944ED
:102E30004160816821448160C1681144C1604022C1
:102E40000021504600F06EF811B000F027B80000E5
:102E5000E599DBE6F87CA21F6556ACC4442229F450
:102E600097FF2A43A72394AB39A093FCC3595B6512
:102E700092CC0C8F7DF4EFFFD15D84854F7EA86FDF
:102E8000E0E62CFE144301A3A111084E827E53F705
:102E900035F23ABDBBD2D72A91D386EB30BCBDE820
:102EA000C08F2DE9F0410F46016905461646C1F372
:102EB000C50001EBC6012961B1EBC60F696901D2FA
:102EC000491C696101EB5671C0F140046961A64279
:102ED00016D3284422463946183000F01AF805F176
:102EE00018012846FFF76AFC04E039192846FFF765
:102EF00065FC403404F13F00B042F6D3002000E00E
:102F00000024321B39192844BDE8F0411830AFF3D2
:102F1000008010B5002302E0CC5CC4545B1C9342DB
:102F2000FAD310BD0023C9B201E0C1545B1C934227
:102F3000FBD370470F4810B50D49016001210171A5
:102F4000417148F2050282600822C2604FF6FF72AA
:102F5000026120224261802282610162FDF7EEFC63
:102F6000002803D0BDE81040FDF7D6BB10BD00001F
:102F700000300240600A00200D4808B5816C41F025
:102F800001018164806C002200F0010000900521A5
:102F90000E20FEF7CDF80E20FEF7BCF8002205212A
:102FA0000F20FEF7C5F8BDE808400F20FEF7B2B8C5
:102FB0000010024010B509A001F02CF80D4A0021C4
:102FC0000D4801F029FC0D4C0A4A002120602432F2
:102FD0000B4801F021FC606010BD0000204D585FDF
:102FE0004652454552544F535F496E697420200D37
:102FF0000A0000009C5F00083135000874000020C2
:103000006D35000870B586B014216846FDF799F952
:103010003448C16C41F00401C164C16C01F0040189
:103020000591C16C41F08001C164C16C01F0800167
:103030000591C16C41F00101C164C16C01F0010155
:103040000591C16C41F00201C164C16C01F0020143
:103050000591C16C41F00801C164C06C224E00F0C2
:103060000800059000220F213046FDF7CAFF4FF6F9
:10307000C0700325CDE9000500246946029430465E
:10308000FDF7E2FE0F2000900120CDE90104694622
:1030900030460394FDF7D8FE49F6FF10CDE9000550
:1030A000694602944FF09040FDF7CEFE4FF6FF7058
:1030B000CDE90005694602940C48FDF7C5FE0420E1
:1030C000CDE90005694602940948FDF7BDFE0820D8
:1030D000CDE90005694602940648FDF7B5FE06B045
:1030E00070BD0000001002400008004800040048C5
:1030F000000C0048001C004870B5224C204820609D
:1031000021480068C1784FF41650082907D2DFE83B
:1031100001F0060406272A2D30334FF4965000257F
:10312000C4E901050C20E560C4E90450A561E5612E
:10313000256214486562FFF76DF808B1FDF7ECFAF7
:10314000124800F110010573416000F5A87181601B
:10315000058045802068016841F01001016070BD64
:103160004FF49640DBE74FF41640D8E74FF4614048
:10317000D5E74FF4E130D2E74FF46130CFE70000FC
:1031800000380140540C002040000020840A002038
:103190000D4810B50B4901604FF4E1314160002149
:1031A00081600C22C160C0E904128161C1610162C9
:1031B0004162FFF72FF8002803D0BDE81040FDF76B
:1031C000ABBA10BD00480040D80C0020FEE700005C
:1031D00070B5144A144C506820601188218192689F
:1031E00062608022A28100226281A273022911D929
:1031F0000E4A126893780278934201D0FF2A09D1CF
:103200004218891E32F8025C01F082FAA84201D10C
:1032100001F0AAFA2089002803D0BDE8704001F02F
:103220008BBF70BD840A00203001002040000020C8
:1032300001F082BFFEE700002DE9F041434E054654
:103240008846F0680024810728680ED0F16801F0F4
:103250000301814207D130B1F0686968C0F3021000
:10326000401C88421FD001246DE0012809D00228AB
:103270000AD00328F7D13168890309D4316849039A
:1032800004E03168890701E0316849050029EADA7C
:10329000F1686A686FF00F0321F0730103EB02120B
:1032A00011430143F160306820F080603060FDF729
:1032B000ADFE074604E0FDF7A9FEC01B022838D882
:1032C00030680001F7D474BBB8F1000F18D0B8F122
:1032D000010F1DD0287D4FF07E41400801EB40607A
:1032E000A96840EA01203169194A11400843306158
:1032F000306840F080603060FDF788FE07461AE0D5
:10330000A868297B000240EAC1603169114AECE7F4
:10331000288A1149400801EB4050A96840EA012081
:1033200031690E4AE1E70EE0FDF770FEC01B02288E
:1033300001D9032407E030680001F5D51CB93069D4
:10334000A969084330612046BDE8F08100100240C1
:10335000FF80FFF9FF80FF070000E0FFFF809FFF75
:10336000F8B51C4E05460024B06DC00002D5FDF72F
:1033700045FF0DE0B06D40F08050B065B06D00F0DD
:1033800080500090FDF73AFFB16D21F08051B1659A
:10339000B0F5007F04D0802D07D94FF003040AE078
:1033A000802D08D9A02D01D804E001D1022402E02B
:1033B000702D00D101240848016821F00701214344
:1033C0000160006800F00700A04201D00120F8BDB4
:1033D0000020F8BD0010024000200240022901D266
:1033E0000020704700210170024909688978417006
:1033F0000220704740000020022901D200207047BF
:103400000021017002490968C978417002207047A3
:1034100040000020042901D2002070470A490A68B0
:10342000D2F8F020120E02700A68D2F8F020120CC6
:1034300042700A68B2F8F020120A8270096891F8A6
:10344000F010C1700420704740000020022901D212
:103450000020704705490A68B2F8EE20120A02708F
:10346000096891F8EE10417002207047400000207A
:1034700010B5102901D2002010BD0C4B002153F8CB
:103480002120120E00F8212053F82120140C00EB0B
:103490008102547033F82140240A947013F82140BB
:1034A000491CD4700429EADB102010BD4400002020
:1034B000022901D20020704705490A68B2F8EC20C1
:1034C000120A0270096891F8EC10417002207047EE
:1034D0004000002010B5FDF7C7F9002010BD000026
:1034E000F0B585B000240494FDF79AFC20200290EA
:1034F0000120CDE9004003900B4D04A96846FDF77B
:10350000BFFB0A4E05EBC40106EBC400D0E9002363
:103510000020FDF72FFC641C0746212CF2D3FDF799
:103520001FFC05B03846F0BD00000108480100202E
:103530000024084E4FF4FA75284601F04BFF012194
:103540003046FDF756FD214603A000F063FD641CE4
:10355000F2E700000008004874686520636F756E2C
:10356000743A205B25645D200D0A0000FFF760FEC1
:10357000064C4FF4FA75FFF72BFE02212046FDF7AB
:1035800038FD284601F00CF9F5E700000008004876
:103590002DE9F04F85B05248002404940068DFF80C
:1035A0004491B0F8FC1001F64521B1F5C0417CD042
:1035B00001F61131B1F5C04F78D1D0F8F810B1F55E
:1035C000803F71D8484F3846FCF738FF00286BD051
:1035D0004348DFF8188100250068A246BB46D0F8B2
:1035E000F8604FF4006296422CD305EB0B013F4884
:1035F000FCF78EFEFDF714FC4F46E819CDF800A04D
:10360000FDF73EF9029001200190039004A968465D
:10361000FDF736FB0024B94608EBC40005EBC401F6
:10362000D0E9002349440020FDF7A4FB641C0746B1
:10363000FF2CF1DDFDF794FB05F50065B6F500669E
:10364000CFD12AE0324605EB0B012848FCF760FE9B
:10365000FDF7E6FB05EB0900CDF800A0FDF710F93A
:10366000029001200190039004A96846FDF708FB31
:1036700000240746F61D0BE008EBC40005EBC4016F
:10368000D0E9002349440020FDF774FB0746641C81
:10369000B4EBD60FF0D3FDF763FB2FB910480068E9
:1036A000D0F8F810C0F8F41001E008E015E00C487C
:1036B00045F2BB510068A0F8FC10FFF711FF084865
:1036C0000068D0F8F410B1F5803F06D84846FCF702
:1036D000B5FE002801D0FFF71FF805B000F008B8CC
:1036E00040000020000002080000030850020020F3
:1036F00030BCBDE8C08F10B54FF0E020006902F08B
:103700009DFA012803D0BDE8104001F0C1BF10BDF3
:1037100010B596B044216846FCF713FE142111A899
:10372000FCF70FFE4FF40070FDF734FD08B172B6E0
:10373000FEE701210804CDE90010022003240A90CD
:10374000CDE90B4114210D910721CDE90E10109008
:103750006846FDF7F3FF08B172B6FEE70F20CDE92A
:1037600011040020139014901590042111A8FDF766
:10377000A7FE002801D072B6FEE716B010BD00000B
:103780000248016841F470010160704788ED00E073
:103790000148FEF7DCBA0000EC0D0020F0B502682D
:1037A000164C4FF08047A04201D0B84203D122F01E
:1037B00070034A681A43124D124EA04205D0B84217
:1037C00003D0A84201D0B04203D122F44073CA68AA
:1037D0001A434B6922F080021A4302608A68C2626F
:1037E0000A688262A04203D0A84201D0B04201D14F
:1037F0000969016301214161F0BD0000002C014015
:1038000000400140004401402DE9F0410D4681781F
:103810004FF6FF7202EA0121C278214C11448FB2A7
:10382000E288E168412300268B54521C92B22B1F80
:103830008E54521C92B2E280B3F5807F01DD0220EB
:1038400004E0B4F804C0674504D004208854521C36
:10385000E2800AE099B2001DFEF7F6FE40B1E08872
:10386000E26808211154401CE080FEF7B5FE0BE031
:10387000E088E1680E54401CE080A0682844001FE6
:10388000A060A088401CA080A188E088E2680B0AA4
:103890001354401C80B21154401CE080BDE8F081FC
:1038A0005400002070B5164C41220025E088E168E4
:1038B0000A54401C80B20D54401CE080FEF78CFE80
:1038C00008B1082104E0A169A068884206D003215C
:1038D000E088E2681154401CE08070BDE088E26836
:1038E0001554401CE0800748006840F8F81F4AF66D
:1038F000AA218180FFF7F4FD0120207070BD000037
:10390000540000204000002090F82410C90706D081
:1039100001684A68836A22F400321A434A6090F8C8
:103920002410890706D501684A68C36A22F48032E8
:103930001A434A6090F82410490706D501684A687E
:10394000036B22F480221A434A6090F8241009077E
:1039500006D501684A68436B22F400421A434A6064
:1039600090F82410C90606D501688A68836B22F492
:1039700080521A438A6090F82410890606D501689F
:103980008A68C36B22F400521A438A6090F82410AC
:10399000490611D501684A68036C22F480121A4363
:1039A0004A60016CB1F5801F06D101684A68436C1A
:1039B00022F4C0021A434A6090F82410090606D582
:1039C00001684A68806C22F4002202434A60704712
:1039D000F8B500250446C0F88050FDF717FB0746F0
:1039E000206800686FF07E46000708D53B4600223D
:1039F0004FF400112046009600F03EFA60B92068AE
:103A0000006840070AD53B4600224FF4800120465B
:103A1000009600F031FA08B10320F8BD2020A0671D
:103A2000E067256684F874500020F8BD10B5806A00
:103A30000021A0F85A10A0F85210FEF7A0FA10BD0D
:103A400070B5846AA06FE56F216889684FF0000641
:103A5000090606D5212804D1A4F85260204600F0BA
:103A6000AEF820688068400606D5222D04D1A4F85F
:103A70005A60204600F07EF8D4F8800040F0100034
:103A8000C4F880002046FEF77AFA70BD10B50146F2
:103A9000806A0968096889062DD40021A0F85A10A7
:103AA000016851E8002F22F4807241E80023002BC6
:103AB000F6D10168083151E8002F22F0010241E8F7
:103AC0000023002BF5D10168083151E8002F22F0C6
:103AD000400241E80023002BF5D12021C167016E8F
:103AE000012908D1016851E8002F22F0100241E8B5
:103AF0000023002BF6D1016E012902D0FEF78EFCC7
:103B000010BDB0F85810FEF7F2F910BD10B5806A7C
:103B1000016E012902D0FEF782FC10BDB0F85810EA
:103B20004908FEF7E4F910BD10B50146806A09683E
:103B30000968890616D40021A0F8521001680831DE
:103B400051E8002F22F0800241E80023002BF5D13C
:103B5000016851E8002F42F0400241E80023002BA9
:103B6000F6D110BDFEF706FD10BD10B5806AFEF758
:103B700002FD10BD016851E8002F22F4907241E867
:103B80000023002BF6D10168083151E8002F22F004
:103B9000010241E80023002BF5D1016E012908D173
:103BA000016851E8002F22F0100241E80023002BA9
:103BB000F6D12021C1670021016641667047016886
:103BC00051E8002F22F0C00241E80023002BF6D17B
:103BD00020218167704700002DE9F041044600680C
:103BE0002369A168E66919436369002533431943D2
:103BF000704A0368704E33400B430360206841688D
:103C0000E36821F44051194341602168A069914261
:103C100001D0236A18438B6823F4306303438B601D
:103C2000664B2168664899420DD1D0F8880010F0A3
:103C3000030006D0012845D0022833D0032830D114
:103C400042E001202EE05F4B99420BD1D0F8880072
:103C500010F00C0026D0042824D0082830D00C28DE
:103C60001FD131E0584B99420BD1D0F8880010F0A9
:103C7000300017D0102825D0202821D0302810D18E
:103C800022E091420DD1D0F8880010F4406009D0B4
:103C9000B0F5806F16D0B0F5006F11D0B0F5406F61
:103CA00012D01020494B00264FF4004C91422ED1E7
:103CB00060B1022813D004280BD0082872D10DE07F
:103CC0000220EFE70420EDE70820EBE7FDF7C0FC5A
:103CD00001E0FDF7E1FC030001D164E063466268A6
:103CE00002EB420098425DD8B3EB023F5AD8190E5E
:103CF0001B025008181871410023FCF7D5FA344A0A
:103D0000A0F5407191424DD82168C8604BE0E1694F
:103D10004FF6EF77614527D1092843D2DFE800F05D
:103D2000050811420D4242421000FDF791FC01E0EE
:103D3000FDF7A0FC030004D135E0FDF7ADFCF9E789
:103D400063466068590001EB5001B1FBF0F0A0F14F
:103D50001001B94226D84FF6F0710140C0F342007D
:103D600001432068C1601EE009281BD2DFE800F093
:103D70000508111A0D1A1A1A1000FDF769FC01E066
:103D8000FDF778FC030004D10DE0FDF785FCF9E7B1
:103D90006346606803EB5001B1FBF0F0A0F1100145
:103DA000B94205D9012566662846A666BDE8F081B8
:103DB00080B2A9E700800040F369FFEF00380140BE
:103DC0000010024000440040004800400024F4007D
:103DD000FFFC0F0070B54165A0F85820002504468F
:103DE000C0F880502220E067206FD8B11F49C1621F
:103DF000216F1F4813460863216F1E484863206FD8
:103E00008563666D216832462431206FFCF700FF20
:103E100040B11020C4F8800004F8745F2020A06036
:103E2000012070BD84F87450206940B1206850E8CA
:103E3000001F41F4807140E80012002AF6D120688A
:103E4000083050E8001F41F0010140E80012002A4C
:103E5000F5D12068083050E8001F41F0400140E8EB
:103E60000012002AF5D1002070BD00008D3A000834
:103E70000D3B0008413A00082DE9F0471F469046E7
:103E80000E4604464FF0000A4FF02009089D49E015
:103E9000681C47D0FDF7BAF8C01BA8422AD84DB31A
:103EA0002068016849073DD5C069C043000539D481
:103EB00021684FF400600862206850E8001F21F478
:103EC000D07140E80012002AF6D12068083050E88E
:103ED000001F21F0010140E80012002AF5D1C4F8CA
:103EE0007890C4F87C90C4F8809084F874A0032083
:103EF000BDE8F087206850E8001F21F4D07140E849
:103F00000012002AF6D12068083050E8001F21F086
:103F1000010140E80012002AF5D1C4F87890C4F8F5
:103F20007C90E2E72068C06936EA000004D00020F7
:103F30004045ADD00020DBE70120F9E70B4810B584
:103F40000068C169C1F3001159B11021016207482D
:103F5000FDF7CFFF0648006840680649C0F5A0702D
:103F60000880BDE810400148FEF70AB8540C002054
:103F70005C0D0020840A0020FEE70000022901D029
:103F80001020704702494078096888700120704706
:103F900040000020022908D14078411E062904D89B
:103FA00003490968C870012070471020704700005D
:103FB00040000020042901D0102070470188827839
:103FC00049BA0904C07841EA022101430248006865
:103FD000C0F8F0100120704740000020022901D0F5
:103FE0001020704703490088096840BAA1F8EE0024
:103FF0000120704740000020022901D010207047A6
:1040000003490088096840BAA1F8EC000120704714
:10401000400000200FB4054B10B503A9044A0298D4
:1040200000F03AF810BC5DF814FB0000F541000800
:104030002C0100200907090E002804DB00F1E02014
:1040400080F80014704700F00F0000F1E02080F8C5
:10405000141D7047BFF34F8F05480168054A01F4EE
:10406000E06111430160BFF34F8F00BFFDE7000027
:104070000CED00E00400FA0502E008C8121F08C1B8
:10408000002AFAD170477047002001E001C1121FD9
:10409000002AFBD1704700002DE9FF4F89B09B46F5
:1040A0000446002506E025280BD05A460B99904778
:1040B000641C6D1C20780028F5D10DB0284600F056
:1040C00095B80027B8460122474900E0074314F895
:1040D000013F203B02FA03F00842F7D120782E2856
:1040E00019D114F8010F47F004072A280ED06FF0F9
:1040F0002F022078A0F1300109290CD808EB8801A3
:1041000002EB410100EB0108641CF2E70A98641C11
:1041100050F8048B0A9020780028CED0642808D06C
:10412000692806D075281ED05A460B9990476D1CF9
:1041300058E00A994FF00A0901C90A91002802DAE9
:1041400040422D2102E0390504D52B218DF82010A5
:10415000012103E0F90704D02021F7E78A4608AEE1
:104160000DE00021FAE70A994FF00A0901C90A9106
:10417000F7E74946FCF7FDF8303106F8011D002845
:10418000F7D1ADEB060000F12009780701D44FF01C
:104190000108C84502DDA8EB090000E000208046C8
:1041A000002706E008A85A46C05D0B9990476D1C91
:1041B0007F1C5745F6DB04E030205A460B999047A8
:1041C0006D1CB8F10001A8F10108F5DC05E016F856
:1041D000010B5A460B9990476D1CB9F10001A9F1EA
:1041E0000109F4DC641C65E70928010030BCBDE866
:1041F000C08F000013B54FF6FF73012269460248D5
:10420000FEF70EF900981CBDD80C0020FCF70CFF3F
:10421000FFF77EFAFCF798F9FFF7BAF9FEF7F2FE1E
:10422000FEF7AAFEFEF768FFFEF7B2FFFEF782FE7A
:1042300000F0C4FAFEF7BEFE00F0D2FAFEE700007E
:104240002DE9F041764D4FF6FF72032629688888E4
:1042500040BA02EA400468680A78027049784170FE
:104260000021817029462A8A8989C91E0B2A7DD09E
:1042700005DC5AB1082A47D0092A04D18EE0102A59
:1042800075D0112A74D00220A8735AE0102C06D0E1
:10429000122C09D0162C15D0182C24D032E089B25B
:1042A000C01CFFF7E5F848E089B2C01CFFF7E0F852
:1042B000C01C87B2A889C01B81B268683844FFF768
:1042C000F7F80EE089B2C01CFFF7D2F8C01C87B225
:1042D000A889C01B81B268683844FFF7E9F8384400
:1042E00053E038442AE089B2C01CFFF7C1F8C01C73
:1042F00087B2A889C01B81B268683844FFF7D8F834
:1043000038440CE0AE731CE0022C12D0062C37D0DF
:10431000082CF7D189B2C01CFFF7CAF8C01C87B2BD
:10432000A889C01B81B268683844FFF773F8384425
:104330003DE089B2C01CFFF7BBF8C01CA97B80B26E
:10434000F1B36868417841F080014170A97B8170C8
:104350006E816989686800F0DBF969896A68505480
:10436000491C89B2000A5054491C02E02EE034E096
:104370004AE089B26981BDE8F041104600F0E8BE2C
:1043800089B2C01CFFF794F8C01C87B2A889C01B73
:1043900081B268683844FFF73DF8A2E7042C10D0DA
:1043A000062CAFD189B2C01CFFF734F8C01C87B20D
:1043B000A889C01B81B268683844FFF747F890E7C6
:1043C00029E089B2C01CFFF725F8B6E7022C99D185
:1043D00089B2C01CFFF73AF8AFE7022C0FD0042CCB
:1043E00090D189B2C01CFEF7F9FFC01C87B2A88922
:1043F000C01B81B268683844FEF7FEFF71E789B2DE
:10440000C01CFEF7EBFF98E7022CCAD189B2C01C92
:10441000FEF7F2FF91E769688C70688199E7000008
:104420003001002070B5354D0024D5E900102A89EF
:10443000FBF76EFF288A032608380A2837D2DFE800
:1044400000F0053636102E30363619222889082815
:1044500005D128680221001DFFF7CEFD1BE0AE73D9
:1044600027E028890828FAD128680221001DFFF7D3
:10447000B5FD10E028890828F1D128680221001D27
:10448000FFF77CFD07E028890828E8D12868022189
:10449000001DFFF77FFD04461028E0D004E0022451
:1044A00002E0FFF717F80324A87B10B301E0022015
:1044B000A8736868417841F080014170A97B8170E0
:1044C00031466E8100F024F969896A685054491CAC
:1044D00089B2000A5054491C69816989686800F0F2
:1044E00037FEE00701D0FEF7FBFFA00704D5FFF77A
:1044F000B1FD28896881F0E770BD0000300100201F
:104500002DE9F0415C4F002439683A8988888D791B
:1045100046BA7868FBF7FCFE30460326B5EB400F41
:1045200004D13889A0F10901A94201D0BE737DE010
:10453000B97B00297AD1398A08390A2974D2DFE88F
:1045400001F00530734B737373735369082D09D0F1
:10455000062D18D00828E9D138680221C01DFFF7C0
:104560004BFD27E038680221C01DFFF745FD0446DA
:10457000386804210930FFF71DFD40EA040538685A
:1045800002210D3025E038680221C01DFFF734FDFF
:104590000546386804210930FFF70CFD40EA0504A0
:1045A00009E0062D0CD0042DC0D138680421C01DAF
:1045B000FFF700FD0446E006B8D4B87B90B335E0C1
:1045C00038680421C01DFFF7F5FC05463868022154
:1045D0000B30FFF703FDE1E7022DA7D13868022178
:1045E000C01DFFF7FBFCE5E7042D07D0022D9DD190
:1045F00038680221C01DFFF7C1FCDBE738680221E3
:10460000C01DFFF7BBFC0546386802210930FFF7E3
:10461000B5FCC3E7022D89D138680221C01DFFF720
:10462000B9FCC7E723E0FFE70220B8737868417858
:1046300041F080014170B97B81707E817989786811
:1046400000F066F879897A685054491C89B2000AEA
:104650005054491C89B27981104600F079FDE00779
:1046600001D0FEF73DFFA00704D5FFF7F3FC0620BD
:104670007881E3E7BDE8F0813001002070B5224D7C
:104680000024D5E900020168116004216981298AAA
:10469000A1F52A43BB3B02D00220A87310E0298970
:1046A000001D891F89B2121DFDF768FF6989084442
:1046B000688116480078012800D10224A87B40B107
:1046C0006868417841F080014170A97B81700320C6
:1046D00068816989686800F01BF869896A685054C4
:1046E000491C89B2000A5054491C89B2698110469C
:1046F00000F02EFDE00701D0FEF7F2FEA00701D585
:10470000FFF7A8FC70BD000030010020540000201D
:104710000A4610B501460248FCF7E9F880B210BD20
:10472000600A002010B50F4CD4E900100968016040
:10473000417841F080014170012181700321618144
:10474000FFF7E6FF618962685054491C89B2000A8C
:104750005054491C89B26181BDE81040104600F0F8
:10476000F7BC0000300100200C4A11684878D07373
:104770004988032849BA118207D0062807D0102893
:1047800007D0422807D0FFF7CDBFFFF759BDFFF78D
:1047900049BEFFF7B5BEFFF771BF00003001002032
:1047A00010B5EFF3058111B16FF0050403E00024AB
:1047B00008B100F00FFE204610BD0000EFF30580A9
:1047C00010B16FF0050070470448016811B14FF057
:1047D000FF3070470121016000207047FC0000207D
:1047E00010B5EFF3058010B16FF0050010BD08485B
:1047F0000168012902D04FF0FF3010BD054A0021A9
:1048000082F8141D0221016000F04CFE002010BD52
:10481000FC0000200BE000E02DE9FF410B464FF0CB
:104820000005EFF30581039549BB40B380261821AD
:1048300000244AB3176807B13C46976907B1394667
:104840004F1E382F02D21779FF0703D0002004B083
:10485000BDE8F081576907B1BE08D2F808C0BCF1C5
:10486000000F0DD0D5685C2D18D312693AB137B15D
:104870008DE806103246214601F0B2F903900DE0B2
:10488000D7685FB912694AB903AACDE90012B2B27A
:10489000214601F075F9012800D003950398D6E769
:1048A0002DE9F041134E0F460446F5683068001DAF
:1048B00000F05EFC601C07D137B13168BDE8F04103
:1048C0000D48091D00F0A4BC30682C44AC42446083
:1048D000316805D2B06BBDE8F041091D00F080BC25
:1048E000706B091D00F07CFCB06A844200D2B46297
:1048F000BDE8F081AC000020281300202DE9F04134
:10490000054600F091FC2D4EB068401CB060306848
:104910002B4F10B1706930B32BE03560B0680128BF
:1049200027D1002404EB840007EB800000F04AFC50
:10493000641C382CF6D3234800F044FC2148143082
:1049400000F040FC1F48283000F03CFC1D483C3083
:1049500000F038FC1B48503000F034FC19487063FC
:104960001430B06305E03068E96AC06A884200D854
:104970003560706A401C70626864E86A3169884218
:1049800000D9306100EB800007EB8000291D00F0AA
:104990003FFC00F069FC706900280CD03068E96ABF
:1049A000C06A884207D208494FF080500860BFF3C0
:1049B0004F8FBFF36F8FBDE8F0810000AC00002087
:1049C000780E0020D812002004ED00E038B500F089
:1049D0002BFC104C2068C8B90F4800F0F3FB0E48C0
:1049E000143000F0EFFB0C48E060143020610A4BFB
:1049F0000020F03B009003F1500210210A2000F04B
:104A00005DFE206010B105A100F0B0FCBDE83840AB
:104A100000F02ABCE80000202C140020546D7251D4
:104A20000000000030B4026C0B46002A0BD0C168B5
:104A30001144C1608468A14201D30168C16030BCE7
:104A40001846FBF765BC30BC70472DE9F041856B1B
:104A5000174604460026026C82B1C7B1E068FBF736
:104A600057FCE168206C091AE1602268914202D289
:104A7000A168081AE060022F16D017E02068A8B9D4
:104A8000A06801F053F906460020A0600EE06068BF
:104A9000FBF73EFC216C606808446060A1688842B6
:104AA00004D32068606001E005B16D1E6D1CA56334
:104AB0003046BDE8F08110B5044690F8590058B171
:104AC00001280CD002280FD0502080F31188BFF3AA
:104AD0004F8FBFF36F8FFEE7206B00F0D9FB2046AE
:104AE000BDE8104000F0D4BB10BD000010484FF4EA
:104AF000FA51420706D0C01D0D4920F00700411AA7
:104B0000C1F5FA510B4A00230144C2E900030839F8
:104B1000183A21F0070111604B600B600B1AC0E9D5
:104B2000001393604FF000405360506170470000E5
:104B30000C1B002018010020134E144DA6F29C47B8
:104B40004FF08058DFF8489011E000F06DFBF068FE
:104B5000C468201D00F00CFBA868401EA8606868AF
:104B6000401E686000F080FB2046FFF7A4FF6868E5
:104B70000028EAD138680128F9D9C9F80080BFF3C4
:104B80004F8FBFF36F8FF2E714130020AC000020AB
:104B900004ED00E070B51D46049C49B12260C4E9F3
:104BA0000F010121204600F0BDFD84F84C5070BD7E
:104BB0002460F4E72DE9F05F0E46DDE90B9417461B
:104BC000834691009A460A9DA522206BFBF7B2FB13
:104BD0006FF00301206B01EB8701084420F0070709
:104BE000780707D0502080F31188BFF34F8FBFF3B1
:104BF0006F8FFEE74FF0000866B100202218315C8D
:104C000082F83410315C11B1401C1028F6D384F8BE
:104C1000438001E084F83480382D00D33725E562E5
:104C2000C4E91358201D00F0D8FA04F1180000F070
:104C3000D4FA2461C5F138006462A061C4F85480DC
:104C400084F8588052465946384600F05FFA206092
:104C5000B9F1000F01D0C9F8004000F000B830BC35
:104C6000BDE8C09F30B5114900E011460A68824294
:104C7000FBD34B685C18844203D1406818444860F9
:104C8000084643681C18944209D1084C183C246813
:104C9000A24209D052681A4442600A68126802604F
:104CA000814200D0086030BD0460F9E7180100209F
:104CB00070B5002441600B4D0061914206D8D11AB5
:104CC0008269914206D2011D286907E09A4203D207
:104CD000994201D3012403E0011DE86800F080FA45
:104CE000204670BDE800002010B5044600F09CFA94
:104CF000A06B20B1002400F0B7FA204610BD0124BB
:104D0000F9E7000030B587B03C4D6EE0019800280F
:104D100006DADDE90301029A90470198002864DB76
:104D2000039C606910B1201D00F022FA05A800F074
:104D3000D7F8024601980A2857D2DFE800F00505A7
:104D4000052D334A05052D3394F8280040F0010065
:104D500084F828000298A169034601442046FFF721
:104D6000A7FF68B3216A2046884794F828004007C7
:104D70003BD5002000900298A169002342181946F3
:104D8000204601F0D9F8D8B9502080F31188BFF33C
:104D90004F8FBFF36F8FFEE714F8280F20F001004C
:104DA000207022E094F8280040F0010084F82800E8
:104DB0000298A06128B1811813462046FFF778FFBA
:104DC00013E0502080F31188BFF34F8FBFF36F8F34
:104DD000FEE794F82800810703D4204600F058FA33
:104DE00003E020F0010084F82800002201A92868CF
:104DF00000F0F0FD002889D107B030BDE8000020A8
:104E00002DE9FC410F46054600F08EFB01A800F09D
:104E100067F80446019818B100F0FEFFBDE8FC8178
:104E2000254EAFB130690068D0B30027291B3A4640
:104E3000306800F0ADFA00F0EFFF0028EED11F4916
:104E40004FF080500860BFF34F8FBFF36F8FE5E7DF
:104E5000A542EBD800F0E0FFF0682746C068C468C0
:104E6000201D00F085F994F82800410719D5A069A4
:104E70002B4641193A462046FFF71AFFA8B10020F9
:104E80000346014600902A46204601F055F860B9D5
:104E9000502080F31188BFF34F8FBFF36F8FFEE771
:104EA00007E020F0010084F82800216A20468847A6
:104EB000B4E70127BAE70000E800002004ED00E0B5
:104EC0000648416B096829B1416BC968C9684968DE
:104ED000816270474FF0FF31FAE70000AC0000201C
:104EE00070B5054600F0B8FE064E0446B068844230
:104EF00003D200F009F8012000E0002028602046DD
:104F0000B46070BDE8000020F8B5194E20E0C0681C
:104F1000C4680568201D00F02BF9216A20468847E7
:104F200094F82800400713D5A0692844A84206D960
:104F300024616060211DF06800F052F908E0002053
:104F40000346014600902A46204600F0F5FF38B19E
:104F5000F06801680029DAD13169C6E90310F8BDAB
:104F6000502080F31188BFF34F8FBFF36F8FFEE7A0
:104F7000E800002008484068401C4FF0500080F3D3
:104F8000118804D0BFF34F8FBFF36F8FFEE7BFF3DD
:104F90004F8FBFF36F8FFEE720010020084CE068C1
:104FA000016839B1002139B10020FFF729FFFFF76F
:104FB000A9FEF4E70121F6E7C0680068F5E7000004
:104FC000E80000202DE9F041044600F02DF994F9A5
:104FD000455004F1240609E0606A48B1304600F00B
:104FE000E3FE08B100F024FA6D1E6DB2002DF3DC73
:104FF0004FF0FF3684F8456000F036F900F014F900
:1050000094F9445004F1100709E0206948B138468A
:1050100000F0CAFE08B100F00BFA6D1E6DB2002D53
:10502000F3DC84F84460BDE8F04100F01DB90000F5
:105030002DE9F0410546002600F076FA324F386837
:1050400008B9FFF753FD786905424ED1C5B308355D
:1050500068070ED005F00700C0F108000544680796
:1050600007D0502080F31188BFF34F8FBFF36F8FAD
:10507000FEE72DB37868854237D8234918310846B2
:10508000046801E0214604466068A84202D2206814
:105090000028F7D13868844227D00E68206808605D
:1050A00060680836411B10290FD96019420708D0E3
:1050B000502080F31188BFF34F8FBFF36F8FFEE74F
:1050C00013E041606560FFF7CDFD61687868401AC4
:1050D0007860BA68904200D2B860786901430020D5
:1050E000C4E90001F868401CF86000F095FE700704
:1050F00007D0502080F31188BFF34F8FBFF36F8F1D
:10510000FEE73046BDE8F0810001002010B5031F26
:105110004FF080741C601B1F21F001011960191FE2
:10512000044B0B6014390A60091F6FF00202443807
:105130000A6010BD754F0008044800214FF4A072AA
:105140000180416800F5E870FDF73EB9840A00204F
:105150000A4610B501460548FDF7BCF9002803D002
:10516000BDE81040FBF7D8BA10BD0000540C002079
:10517000D0E9013201699A60D0E901235A604A6896
:10518000824201D182684A60002202610868401EA2
:105190000860086870470000034B036003F15C007F
:1051A000086080201060704754140020044B036096
:1051B00003F15C0008604FF48070106070470000DD
:1051C000B016002000F108014FF0FF32C0E90112D3
:1051D000C1600161002101607047002101617047D9
:1051E00030B50C68621C02D000F1080202E00269CE
:1051F00004E01A4653681D68A542FAD953684B600B
:1052000099608A60516008610168491C016030BD85
:1052100042684A6093688B60936859609160086146
:105220000168491C01607047502080F31188BFF36A
:105230004F8FBFF36F8F0A494868401C48600128B0
:105240000CD10848006810F0FF0F07D0502080F301
:105250001188BFF34F8FBFF36F8FFEE770470000D9
:105260002001002004ED00E00849486828B1401EF4
:10527000486001D180F311887047502080F3118875
:10528000BFF34F8FBFF36F8FFEE7000020010020B8
:1052900070B500282AD0164DA0F10804606869692D
:1052A000084207D1502080F31188BFF34F8FBFF31E
:1052B0006F8FFEE722683AB1502080F31188BFF368
:1052C0004F8FBFF36F8FFEE78843606000F02CF9CB
:1052D00060686968084468602046FFF7C3FC286975
:1052E000401C2861BDE8704000F096BD70BD000014
:1052F000000100204FF0E02000210161816105499B
:105300004FF47A720968B1FBF2F1491E416107213D
:1053100001617047A800002010B5FAF79FFF1149FE
:1053200010280ED300F1E02090F8F0030A789042A4
:1053300007D2502080F31188BFF34F8FBFF36F8FD8
:10534000FEE709480068896800F4E060884207D9F0
:10535000502080F31188BFF34F8FBFF36F8FFEE7AC
:1053600010BD0000200100200CED00E010B5074B3F
:10537000002253F832401CB1521C082AF9D310BD48
:1053800043F8321003EBC201486010BD380E002014
:1053900070B515460E460446FFF746FF94F94410D3
:1053A0000020491C01D184F8440094F94510491C9F
:1053B00001D184F84500FFF757FFA06B28B92A46B2
:1053C000314604F1240000F051F82046BDE8704059
:1053D000FFF7F8BD10B5020014D00F48006B38B1CC
:1053E000502080F31188BFF34F8FBFF36F8FFEE71C
:1053F00000F09AF800211046FFF752FA00F00CFD79
:10540000002807D105494FF080500860BFF34F8F47
:10541000BFF36F8F10BD0000AC00002004ED00E072
:1054200002490A6A0260C96841607047AC00002006
:1054300001490120C8617047AC00002010B50C463E
:1054400050B1094909681831FFF7CAFE2046BDE886
:1054500010400121FFF724BA502080F31188BFF3D8
:105460004F8FBFF36F8FFEE7AC00002070B514467E
:105470000D4668B10A4909681831FFF7C9FE0CB139
:105480004FF0FF3521462846BDE87040FFF708BAC7
:10549000502080F31188BFF34F8FBFF36F8FFEE76B
:1054A000AC00002030B587B00025039505AA04A9FB
:1054B00003A80495FFF770FEDDE903010095CDE92F
:1054C0000110002314A11648059A00F089FB154C21
:1054D000E06218B100F000FD012809D0401C19D18C
:1054E000502080F31188BFF34F8FBFF36F8FFEE71B
:1054F000502080F31188BFF34F8FBFF36F8F4FF0B1
:10550000FF30A06201206061E56007B0BDE8304077
:1055100000F044B807B030BD49444C4500000000DD
:10552000394B0008AC0000200248016B491C0163A4
:1055300070470000AC000020164B10B5186B10B17E
:105540000120D86110BD0020D8611869124901E01E
:10555000B8B1401E00EB800251F82220002AF7D09B
:1055600000EB800201EB820101F108044A685268F5
:105570004A60A24201D152684A60D168196018613C
:1055800010BD502080F31188BFF34F8FBFF36F8F92
:10559000FEE70000AC000020780E00201CB5374864
:1055A0000168374A914207D1502080F31188BFF338
:1055B0004F8FBFF36F8FFEE700683149491E884265
:1055C00007D1502080F31188BFF34F8FBFF36F8F47
:1055D000FEE72C4908780190FF20087008788DF8C4
:1055E00000009DF800009DF8002000F0F0009042BF
:1055F00007D0502080F31188BFF34F8FBFF36F8F18
:10560000FEE79DF80000204C00F0500020700720BD
:10561000A06006E0401EA0609DF8000040008DF8EC
:1056200000009DF800000006A068F3D4032807D00E
:10563000502080F31188BFF34F8FBFF36F8FFEE7C9
:105640004FF44070A060019808700C482030016849
:1056500041F470010160016841F070410160FFF7A1
:1056600049FE00206060FAF7C1FD0848016841F07A
:1056700040410160FAF7A6FD00201CBD00ED00E0EE
:1056800071C20F4100E400E02001002034EF00E08F
:1056900010B5502080F31188BFF34F8FBFF36F8F89
:1056A00000F0E0FA18B104494FF080500860002083
:1056B00080F3118810BD000004ED00E038B5049DB2
:1056C00018B153B1CAB181B120E0502080F31188E4
:1056D000BFF34F8FBFF36F8FFEE7502080F3118829
:1056E000BFF34F8FBFF36F8FFEE7502080F3118819
:1056F000BFF34F8FBFF36F8FFEE739B1502080F3B8
:105700001188BFF34F8FBFF36F8FFEE750241C4605
:10571000012384F846302B460094FFF73BFA2046DD
:1057200038BD000070B50D46040025D0FFF77CFDA4
:10573000D4E90F20216802FB0011A1600021A163C0
:10574000216861600A46D4E90F01401E00FB012177
:10575000E16021464FF0FF3001F8440F487004F13A
:1057600010008DB1FFF72EFD04F12400FFF72AFD94
:10577000FFF77AFD012070BD502080F31188BFF340
:105780004F8FBFF36F8FFEE721690029F0D000F043
:105790000BFB0028ECD004494FF080500860BFF3A9
:1057A0004F8FBFF36F8FE3E704ED00E02DE9FF4F6C
:1057B00083B01F468B4604004FF0000603D0BBF1B8
:1057C000000F08D011E0502080F31188BFF34F8FF5
:1057D000BFF36F8FFEE7206C38B1502080F3118843
:1057E000BFF34F8FBFF36F8FFEE7022F0AD1E06B3D
:1057F000012807D0502080F31188BFF34F8FBFF3EB
:105800006F8FFEE700F01AFADFF800914FF0000A00
:105810004FF0805848B9059838B1502080F311886E
:10582000BFF34F8FBFF36F8FFEE7FFF7FDFCA06B59
:10583000E16B884205D3022F03D00598C8B1DEB1D1
:105840001EE03A4659462046FFF7FFF8616A19B153
:1058500004F1240000F0A8FA28B1C9F80080BFF3D1
:105860004F8FBFF36F8FFFF7FFFC012007B000F0F1
:105870004FB8FFF7F9FC21E06846FFF7D1FD01269C
:10588000FFF7F2FCFFF750FEFFF7CEFC94F944005F
:10589000401C01D184F844A094F94500401C01D17A
:1058A00084F845A0FFF7E0FC05A9684600F02EF952
:1058B00030B12046FFF786FB00F0AEFA0020D5E7B6
:1058C000FFF7B2FCA06BE16B884201D1012500E03B
:1058D0000025FFF7C9FC95B104F110000599FFF709
:1058E000ADFD2046FFF76EFB00F096FA00289CD134
:1058F000C9F80080BFF34F8FBFF36F8F95E7204645
:10590000FFF760FB00F088FA8FE7000004ED00E08D
:1059100030BCBDE8C08F2DE9F0471F469046894650
:10592000040003D0B9F1000F08D011E0502080F33B
:105930001188BFF34F8FBFF36F8FFEE7206C38B134
:10594000502080F31188BFF34F8FBFF36F8FFEE7B6
:10595000022F0AD1E06B012807D0502080F3118874
:10596000BFF34F8FBFF36F8FFEE7FFF7D5FC5020DB
:10597000EFF3118680F31188BFF34F8FBFF36F8F62
:10598000A06BE16B884206D3022F04D0002086F37F
:105990001188BDE8F08794F94550A06B3A46494616
:1059A0002046FFF752F8681C04D06D1C84F845505F
:1059B0000120ECE7606A0028FAD004F1240000F02E
:1059C000F3F90028F4D0B8F1000FF1D00121C8F8A4
:1059D0000010EDE72DE9F74783B08A4604004FF049
:1059E000000603D0BAF1000F08D011E0502080F378
:1059F0001188BFF34F8FBFF36F8FFEE7206C38B174
:105A0000502080F31188BFF34F8FBFF36F8FFEE7F5
:105A100000F014F9DFF8F09000274FF0805848B9F3
:105A2000059838B1502080F31188BFF34F8FBFF332
:105A30006F8FFEE7FFF7F8FBA56BC5B15146204617
:105A4000FEF7F0FF6D1EA563206950B104F1100050
:105A500000F0AAF928B1C9F80080BFF34F8FBFF357
:105A60006F8FFFF701FC012006B0BDE8F0870598B5
:105A700008B11EB106E0FFF7F7FB27E06846FFF725
:105A8000CFFC0126FFF7F0FBFFF74EFDFFF7CCFB45
:105A900094F94400401C01D184F8447094F9450005
:105AA000401C01D184F84570FFF7DEFB05A968466C
:105AB00000F02CF8002820460AD0FFF783FA00F007
:105AC000ABF92046FFF710F90028B3D00020CBE750
:105AD000FFF70AF990B104F124000599FFF7AEFC35
:105AE0002046FFF76FFA00F097F90028A2D1C9F815
:105AF0000080BFF34F8FBFF36F8F9BE72046FFF708
:105B000061FA00F089F995E704ED00E02DE9F04134
:105B10000C46050011D0C4B1FFF786FB174EF168A3
:105B20006B682268C81A571C17D02F68366AB742AC
:105B300019D08B4217D8012410E0502080F311882F
:105B4000BFF34F8FBFF36F8FFEE7502080F31188B4
:105B5000BFF34F8FBFF36F8FFEE70024FFF784FB87
:105B60002046BDE8F081824205D9101A20602846FF
:105B7000FFF756FCF1E700202060DCE7AC000020D6
:105B80002DE9FF5F8346DDE90E87994616468A4672
:105B90009000FFF74DFA05001CD05C20FFF748FA93
:105BA000040014D00020256384F85900CDE9024098
:105BB000CDE900874B46324651465846FEF7FAFF7C
:105BC0002046FEF79BFE012004B000F006B82846F0
:105BD000FFF75EFB4FF0FF30F6E730BCBDE8C09F3B
:105BE000F0B585B00546DDE90B040A9EA8B1E4B125
:105BF0005C2700972063022084F859000020CDE93B
:105C0000024004AF2846CDE90067FEF7D3FF2046E7
:105C1000FEF774FE049805B0F0BD502080F31188A3
:105C2000BFF34F8FBFF36F8FFEE7502080F31188D3
:105C3000BFF34F8FBFF36F8FFEE700000548416948
:105C400019B1006B18B10020704701207047022085
:105C500070470000AC0000200148C0687047000099
:105C6000AC0000202DE9F0412E4F0026386B28B102
:105C7000B869401CB8613046BDE8F081FD686D1C14
:105C8000FD6013D1786B006838B1502080F3118823
:105C9000BFF34F8FBFF36F8FFEE7786BB96B7963FC
:105CA000B863386A401C3862FFF70AF9B86ADFF84F
:105CB0007880854209D3786B0068A0B1786BC068A2
:105CC000C4686068854211D2B8623868C06A00EB67
:105CD000800158F82100012800D90126F869002820
:105CE000C9D00126C7E74FF0FF30EDE7201DFFF7D1
:105CF0003FFAA06A18B104F11800FFF739FAE06A18
:105D00003969884200D9386100EB800108EB8100D5
:105D1000211DFFF77DFAE06A3968C96A8842CAD353
:105D20000126C8E7AC000020780E002070B5040002
:105D30004FF000002BD01A4D29688C4207D050201C
:105D400080F31188BFF34F8FBFF36F8FFEE7216D94
:105D5000F1B1491E2165E36CE26A9A4217D000292D
:105D600015D1201DFFF704FAE06CE062C0F13800A5
:105D7000A061E06A2969884200D92861094900EBDD
:105D8000800001EB8000211DFFF742FA012070BD69
:105D9000502080F31188BFF34F8FBFF36F8FFEE762
:105DA000AC000020780E002070B5C068C46854B103
:105DB00004F118000646FFF7DBF9144D286B50B1CB
:105DC0003146134815E0502080F31188BFF34F8F00
:105DD000BFF36F8FFEE7201DFFF7CAF9E06A29695C
:105DE000884200D928610B4900EB800001EB80005C
:105DF000211DFFF70DFAE06A2968C96A884202D9B5
:105E00000120E86170BD002070BD0000AC000020E2
:105E100000130020780E00202DE9F0472B4D0024C0
:105E20002746286B38B1FFF7FFF9286B401E28631F
:105E3000286B40B145E0502080F31188BFF34F8FAD
:105E4000BFF36F8FFEE7A86821490126C8B3A1F50B
:105E500091698846D8F80010E1B1D8F80C00C46800
:105E600004F11800FFF784F9201DFFF781F9E06ABB
:105E70002969884200D9286100EB800109EB810083
:105E8000211DFFF7C5F9E06A2968C96A8842E1D394
:105E9000EE61DFE70CB1FFF713F8AC693CB1FFF737
:105EA000E1FE00B1EE61641EF9D10020A861E8694D
:105EB00038B10849012738070860BFF34F8FBFF397
:105EC0006F8FFFF7D1F93846BDE8F087AC000020AE
:105ED0000013002004ED00E010B586B0FEF776FD5B
:105EE000114C2068B8B100200390049005AA04A9C1
:105EF00003A8FFF75BF9DDE9032102208DE8070025
:105F000000230AA10B48059AFFF76AFE606010B1F2
:105F100006B0012010BD502080F31188BFF34F8FD1
:105F2000BFF36F8FFEE70000E8000020546D722081
:105F3000537663009D4F00082DE9FF411F46030083
:105F40000A9E4FF0000015D0134D2C68002C0ED087
:105F50008DE80E00062917DAFFF770FE02284FF0D1
:105F600000030FD0002269462868FFF71FFC04B029
:105F7000BDE8F081502080F31188BFF34F8FBFF34D
:105F80006F8FFEE73246EEE700233A466946204629
:105F9000FFF7C1FCEBE70000E800002038600008D4
:105FA00000000000000000000000000000000000F1
:105FB00000020000180000000000000000000000C7
:105FC0002C6000080000000000000000000000003D
:105FD00000000000000200001800000000000000A7
:105FE00000000000000000000000000001020304A7
:105FF00006070809A0860100400D0300801A06006C
:1060000000350C0040420F0080841E0000093D0056
:1060100000127A000024F40000366E010048E80106
:10602000006CDC0200000000010203044D6F64629A
:1060300075735461736B000064656661756C7454AC
:1060400061736B00646000080000002030010000F4
:10605000000400088460000830010020203D00009A
:1060600088400008024080C648010020010529023E
:10607000FE34014201021810021101037A093D9514
:04608000AAAAAAAA74
:040000050800018D61
:00000001FF
